:040000008A15A02F8E
:10000600831203173B0803139300831614180D2855
:0C0016000000082883121308F000080006
:1000220083120313F801F9011030FC00710DF80D71
:10003200F90D7408F8027508031C750FF90203180C
:1000420029287408F80775080318750FF9070310B3
:0A005200F00DF10DFC0B172808005B
:10005C00831203138710403003173804BB000320AE
:10006C0003173908BB00032003173A08BB00032011
:04007C0087140800DD
:1000800083120317B6010530360203184E283608CE
:100090003507840020308000B60A4328360835072B
:1000A00084008001B60336083507B7000A30F40033
:1000B000F5013308F0003408F10011207808F00051
:1000C0007908F1003030F007031737088400700812
:1000D00080000A30F400F5013308F0003408F10024
:1000E000112070080317B3007108B40000307106C6
:1000F000031D7C2800307006031D7F288128B6036D
:040100005328080078
:1001040083120317B8013308B9003408BA002E204B
:1001140087103A300317BB0003200317BB010320E9
:040124008714080034
:0E0128008316031343088A0042088200080071
:100136000E3083120313FD00FD0B9F2800000800FC
:10014600831203138710803003173304BB00032088
:0C01560003173408BB00032087140800C6
:10016200023083120317B8003308B9003408BA000A
:100172002E2087107A300317BB000320031735089F
:08018200BB00032087140800F4
:10018A00831203138710A03003173304BB00032024
:0C019A0003173408BB0003208714080082
:1001A60083120313871003173308BB0003200317BA
:0801B600BB01032087140800BF
:1001BE008312031387107A300317BB000320031733
:0A01CE003308BB000320871408006B
:1001D800831203172B08F1002C08F2000130AB0240
:1001E800031CAC0300307206031DFC2800307106A6
:1001F80003191729290884000008F1002A08840037
:100208007108000603191429290884000008F00061
:100218002A0884000008F002F101031CF1031929DF
:0C022800A90AAA0AEC28F001F101080064
:10023400831203172908393C031C2729303029026B
:0E024400031C27290130F0002829F0010800D2
:1002520083120317AB01AC01031387107A30031723
:10026200BB00032003172908F000A90A70088400C4
:100272000008F0007008AA007008031948292A082B
:10028200BB0003200317AB0A0319AC0A332903137B
:0E029200871403172B08F0002C08F100080059
:1002A00083120317AC01AD01031387107A300317D3
:1002B000BB00032003172908F0002A08F100A90A4F
:1002C0000319AA0A700883160313C2007108C30039
:1002D00094208A110A12F000700883120317AB00F1
:1002E000700803197B292B08BB0003200317AC0AF5
:1002F0000319AD0A5A290313871403172C08F000B9
:060300002D08F1000800C9
:10030600831203172B082907AD002A080318013E9C
:100316002C07AE000130AD02031CAE031030B8004E
:100326002908B9002A08BA002E2012300317B8008F
:100336002D08B9002E08BA002E201F300317B3006F
:100346003030B400A3201F300317B300D320F01EB3
:06035600AD29A6290800F4
:10035C00023083120317B8002908B9002A08BA0022
:10036C002E2087107A300317BB00032003172C08AC
:10037C002D040319CD292B0884000008BB00032091
:10038C000317AB0A0130AC02031CAD03BC290313E9
:04039C0087140800BA
:1003A000AE3083120317B3001930B400B501B12089
:1003B000AE3003172907F0002A080318013E193E42
:1003C000F1007008A9007108AA000630B800700892
:1003D000B9007108BA002E201F300317B300803017
:1003E000B400A3201F300317B3008030B400C52031
:1003F0006808053A0319012A6808073A0319012A0F
:10040000072A1C300317B3000A30B400C5201F3080
:100410000317B3000830B400A3206808053A031995
:10042000162A6808073A0319162AA32A0317AC01EB
:10043000AD011C30B300D3200A30F0057008031D55
:100440002E2A0317AC0A0319AD0A03302D02031D2F
:100450002B2AE8302C0203182E2A192A03171C30E5
:10046000B300D320F0183E2A033003172D02031DDA
:100470003B2AE8302C0203183E2AA22A03171F3019
:10048000B3000830B400C520043003172907B300B7
:100490002A080318013EB40082207008E700031701
:1004A000AB0110302B020318A22A1C30B300D3205A
:1004B000F01C9E2AE71E9E2A1F300317B3008030CF
:1004C000B400A3201F300317B3008030B400C52050
:1004D0001C300317B3000A30B400C5201F300317C7
:1004E000B3000830B400A3200317AC01AD011C30E9
:1004F000B300D3200A30F0057008031D8C2A0317BF
:10050000AC0A0319AD0A03302D02031D892AE83015
:100510002C0203188C2A772A03171F30B3000830E7
:10052000B400C520043003172907B3002A080318B4
:10053000013EB40082207008E7009F2AA22A031718
:10054000AB0A512AAA2A03171F30B300D320F01D8B
:10055000AA2AA32A1D300317B300D3200630F005C2
:1005600070080319B52AF001B72A0130F00008001D
:1005700083120317AE01AF012908B0002A08B100A9
:1005800080302A06F00080307002031DC92A003036
:1005900029020318D72A0130AE000030AF00290825
:1005A000003CB0002A08031C013EB101B102300832
:1005B000B3003108B4002B08B50040200630AC0071
:1005C0000030AD002D08003C031DE82A2C08003C3B
:1005D0000318032B2C082B07F20001302C02F0002B
:1005E0000030031C013E2D02F10070082B0784002F
:1005F0000008F00072088400700880000130AC022E
:10060000031CAD03E22A2B088400203080002E0852
:100610002F040319212BAC01AD012C082B078400FA
:100620000008203A031D182BAC0A0319AD0A0D2B44
:100630000130AC02031CAD032C082B0784002D30C5
:04064000800008002E
:100644008312031387103A300317BB0003200317E8
:08065400BB010320871408001C
:10065C008312031387107A300317BB000320031790
:10066C002A08F0002B08F1000130AA02031CAB038E
:10067C007008710403194A2B290884000008BB0078
:0E068C0003200317A90A352B03138714080057
:10069A008312031387107A300317BB000320031752
:1006AA002A08BB00032003172908BB00032087146C
:0206BA00080036
:1006BC00831203139F01C0309F0483161F179F17CB
:1006CC00831203172908F000F00D7010F00D701054
:1006DC00F00D7010700803139F041F149B201F153E
:1006EC001F1D7A2B0000762B1F101E08F100F00145
:0C06FC0083161E08F0040030F104080012
:10070800831203172908B3002A08B4002B08B50080
:0C071800B12003172C08B300DF200800FC
:1007240083120317B2010130AB02031CAC032F0880
:100734000319AD2B2C08193C031DA22B2B08AD3C2F
:100744000318AD2BB20AAD302B02B0001930031CD4
:10075400013E2C02B10032080319B52BAD30F10073
:100764001930F200B92B2B08F1002C08F2002A08EA
:100774007206031DBF2B71082906031DCF2B290800
:10078400B3002A08B400822070080317B5002D08AE
:10079400B3002E08B400B120062C10300317B800A3
:1007A4002908B9002A08BA002E2012300317B8000D
:1007B40032080319E22BAD30F0001930F100E62BBA
:1007C4002B08F0002C08F1007008B9007108BA0079
:1007D4002E2014300317B8002D08B9002E08BA00D3
:1007E4002E201F300317B3001030B400C5201F3073
:1007F4000317B3002030B400A3201F300317B30045
:10080400D320F01E062CFF2B0317320803192D2CBE
:1008140029082B02F0002A08031C013E2C02F100D7
:100824003008F002031CF1033108F102F00A031945
:10083400F10A7008AD0771080318013EAE070130D4
:100844003002AB000030031C013E3102AC00A901B0
:08085400AA01B201AD2B08005E
:10085C00023083120313FC004930FD00FD0B342CD5
:0A086C00FC0B342C00000000080013
:10087600AF3083120317A9001930AA001C08AB0079
:100886000630AC000030AD00AE215E300317A90083
:100896000630AA000030AB002E2300300317A90053
:1008A6000830AA004D23031722081C3EA50000307D
:1008B6000318013E2307A6000030A9004530AA0010
:1008C6004D2303172508A9002608AA004D2365080D
:1008D6000317A900031366080317AA004D23E50AA8
:1008E6000319E60A0317A901AA014D2311300317BC
:1008F600A9008030AA004D230317A901AA014D23A0
:1009060069300317A9000430AA000030AB002E237B
:1009160003171D08A9000430AA000030AB002E23DF
:10092600083003172207A50023080318013EA60076
:100936001E08A9001F08AA004D2303172008A900B6
:100946002108AA004D2303172508A9002608AA0096
:100956004D230317A901AA014D23BD300317A90092
:100966001930AA001430AB000030AC0083211630D9
:100976000317B300D32070080317A7001730B3007E
:10098600D32070080317AB00C730A9001930AA009E
:100996002708AC008423013003172505A40022088C
:1009A600D93EB30019300318013E2307B400B50140
:1009B600B120C9300317A9001930AA00D130AB0005
:1009C6001930AC002208D93EAD0019300318013E9B
:1009D6002307AE002408AD070318AE0AAF01922321
:1009E6002208D93EA90019300318013E2307AA00A0
:1009F6002408A9070318AA0A0830A9070318AA0A8F
:100A0600AB011130AC00842303172608B300DF20A6
:100A160003172508B300DF20D1300317A9001930CA
:100A2600AA000C302507AB0026080318013EAC00CF
:100A36002408AB070318AC0A832116300317B3004A
:100A4600D32070080317A7001730B300D32070080F
:100A56000317AB00D730A9001930AA002708AC004D
:100A66008423031722082A3EA90000300318013EFA
:080A76002307AA00D0210800AB
:100A7E00831203171E08FF3A031D472DFF301D0674
:100A8E0003194F2DB8011D08B9001E08BA002E20FB
:100A9E00031387103A300317BB00032003171F08F8
:100AAE00F0002008F10001309F02031CA003700823
:100ABE00710403196B2DBB01032003171C0884005E
:0E0ACE00700880009C0A552D03138714080041
:0A0ADC0083120313F001F10108007A
:100AE60083120317A601A70100302006031D7D2DE2
:100AF60050301F060319822DF001F101672FA40162
:100B0600A50100302502031D8A2D0A302402031890
:100B1600992D24084D3EA800222303172808840097
:100B260070088000A40A0319A50A842D24084D3EE6
:100B3600840080014D30A9003430AA000530AB0096
:100B46000030AC00EC20700871040319AD2DF001E3
:100B5600F101672F03133008F0003108F100320865
:100B6600F2003308F300F00A0319F10A0319F20A36
:100B76000319F30A7008B0007108B1007208B200D8
:100B86007308B3005208DD005208733A031DAD2EF8
:100B960002300317A9001730AA0050217008A600DA
:100BA6007108A700F330A9000F30AA005021700881
:100BB600A60771080318013EA7070230A9005E23A5
:100BC600700883120317A9007108AA00A030AB00B1
:100BD600B8225530A9001730AA0050217008A60780
:100BE60071080318013EA707A030A9002921700843
:100BF600A60771080318013EA7076230A90017303F
:100C0600AA0050217008A60771080318013EA7071D
:100C16000330A9005E23700883120317A900710828
:100C2600AA00A030AB00B8224330A9001730AA00B2
:100C360050217008A60771080318013EA707A030C7
:100C4600A90029217008A60771080318013EA70705
:100C56006030A9001730AA0050217008A607710855
:100C66000318013EA7072D30A9001730AA0050210E
:100C76007008A60771080318013EA7070608A90011
:100C8600AA01A030AB00B822A030A9002921700823
:100C9600A60771080318013EA7076630A90017309A
:100CA600AA0050217008A60771080318013EA7077D
:100CB6003830A9001730AA0050217008A60771081D
:100CC6000318013EA707031308080317A900AA0182
:100CD600A030AB00B822A030A90029217008A607D1
:100CE60071080318013EA7076430A9001730AA004F
:100CF60050217008A60771080318013EA7070313C1
:100D060030080317A900031331080317AA00A030FF
:100D1600AB00B8224C30A9001730AA005021700849
:100D2600A60771080318013EA707A030A9002921CC
:100D36007008A60771080318013EA7075E30A900D0
:100D46001730AA0050217008A60771080318013E43
:100D5600A707192F03135D08643A031D192F5308BB
:100D66000317A9001A2170080319192F303003132D
:100D76005302DC0054086F3A031DC22ECC015408FE
:100D8600663A031DC82E0130CC00F92E4C18CD2E24
:100D96000810CE2E0814192F4C18D32E8810D42ED6
:100DA6008814192F4C18D92E0811DA2E0815192F68
:100DB6004C18DF2E8811E02E8815192F4C18E52EB9
:100DC6000812E62E0816192F4C18EB2E8812EC2E58
:100DD6008816192F4C18F12E0813F22E0817192F02
:100DE6004C18F72E8813F82E8817192F5C08003A2E
:100DF6000319C92E5C08013A0319CF2E5C08023A82
:100E06000319D52E5C08033A0319DB2E5C08043A55
:100E16000319E12E5C08053A0319E72E5C08063A29
:100E26000319ED2E5C08073A0319F32E0030031759
:100E36002706031D202F00302606031D632F0230D0
:100E4600A9001730AA0050217008A6007108A70053
:100E56002130A9001730AA0050217008A607710892
:100E66000318013EA707031322080317A90003135B
:100E760023080317AA0050217008A6077108031853
:100E8600013EA707031320080317A900031321082F
:100E96000317AA0050217008A60771080318013E1F
:100EA600A70703132E080317A90003132F08031718
:100EB600AA0050217008A60771080318013EA7076B
:0A0EC6002608F0002708F1000800DC
:100ED000C93083120317A9001930AA00CD30AB0026
:100EE0001930AC00CD30AD001930AE00AF01922307
:100EF000C930A9001930AA006930AB000430AC0039
:080F00000030AD00AE21080035
:100F0800831203138710403003171C04BB0003200F
:0C0F180003171D08BB000320871408000D
:100F2400831203179C01C8301C0203189E2F2E2421
:0A0F34002E2403179C0A952F0800D5
:100F3E00B53083120317A9001930AA00BB30AB00DD
:100F4E001930AC00AF30AD001930AE00AF019223B6
:100F5E00B530A9001930AA005E30AB000630AC00E7
:080F6E000030AD00AE210800C7
:100F7600831203171D08193C031DC32F1C08AD3C23
:100F86000318CB2FAE309C02031C9D0319309D0223
:0E0F9600B8011C08B9001D08BA002E20080082
:100FA400831603134808F3004708F2004908F000C9
:100FB4004A08F1000130C902031CCA037008710415
:100FC4000319EF2F730884000008F00072088400EE
:100FD40070088000F20AF30AD82F4708F0000800CE
:100FE4008316031387128711071683129401403066
:0A0FF400831694008312941608007F
:1010000083120317B3018A11D3208A1570080317BE
:10101000A0000130B3008A11D3208A15700803178D
:10102000A100B8011C08B9001D08BA008A112E20C1
:101030008A1587103A300317BB008A1103208A15DE
:1010400003171F0803193328BB018A1103208A15CF
:1010500003171E088400700800060319302833287F
:101060009E0A9F032028031387140317B801200842
:10107000B9002108BA008A112E208A1503171F080B
:04108000F000080074
:1010840083160313570883120317B300831603133D
:10109400580883120317B4008A1182208A15700835
:1010A4008316E7008A1122238A1570088316E60046
:1010B4008A1122238A1570088316E5008A112223D7
:1010C4008A1570088316E400EC01EF0101308312E5
:1010D40003179200900191010C30831603135707F4
:1010E40083120317B3008316031358080318013E31
:1010F40083120317B4008A1182208A15700883169C
:10110400EA00EB01EA0CEA13EA0CEA130030EB0004
:10111400FC30EA05FF30EB05BE30831203179C0058
:10112400C9309D0019309E0004309F000030A0009B
:101134008A113F258A150D3083165707831203172A
:10114400B3008316031358080318013E83120317D0
:10115400B4008A1182208A153F3070058316E80096
:10116400E9010030E9050030E9000E3083126D0218
:101174008316ED000030031C013E83126E028316B9
:10118400EE005508ED02031CEE035608EE026A0851
:10119400ED02031CEE036B08EE02023057078312C4
:1011A4000317B3008316031358080318013E831270
:1011B4000317B4008A1182208A1570080317B5003A
:1011C40083160313570883120317B30083160313FC
:1011D400580883120317B4008A11B1208A1503300A
:1011E4008316570783120317B30083160313580893
:1011F4000318013E83120317B4008A1182208A1552
:1012040070080317B3008A11DF208A158316660855
:1012140083120317A90083160313670883120317A5
:10122400AA008A114D238A150430831657078312A6
:101234000317B3008316031358080318013E8312DF
:101244000317B4008A1182208A15700803179600C8
:101254008A1122238A157008031795008A11222304
:101264008A157008031794008A1122238A157008BE
:10127400031793008A1122238A15700803179A0012
:101284008A1122238A157008031799008A112223D0
:101294008A157008031798008A1122238A1570088A
:1012A400031797000030831603136906031D5C2996
:1012B40002306806031DAC29831203171308F000DB
:1012C4001408F1001508F2001608F300F00A0319D7
:1012D400F10A0319F20A0319F30A70089700710856
:1012E40098007208990073089A0012308316031349
:1012F400E8000030E9000C3083120317B3008A11B0
:10130400D3208A157008031793000D30B3008A1197
:10131400D3208A15700803179400B3018A11D320CF
:101324008A157008031795000130B3008A11D32081
:101334008A1570080317960083160313EC0A1830F5
:10134400EA000030EB0083120317900191010313AC
:10135400CB015E2A003083166906031DB3291830B9
:101364006806031D042A8312031713088316031344
:10137400D90083120317140883160313DA008312A7
:101384000317150883160313DB00831203171608CB
:1013940083160313DC00831203171708930018083D
:1013A4009400190895001A089600831603136D0813
:1013B400F0006E08F100F201F3015908F0075A0831
:1013C40003185A0FF1075B0803185B0FF2075C0858
:1013D40003185C0FF3077008831203179700710852
:1013E40098007208990073089A001030831603134A
:1013F400E8000030E900EC0A1430EA000030EB00A9
:10140400EF0A5E2A00306906031D0A2A11306806B5
:10141400031D5E2A83120317130883160313DD00CA
:1014240083120317140883160313DE0083120317B1
:10143400150883160313DF00831203171608831697
:101444000313E0008312031717089300180894008D
:10145400190895001A089600831603135D08F00016
:101464005E08F1005F08F2006008F300F00A031957
:10147400F10A0319F20A0319F30A70088312031715
:101484009700710898007208990073089A00103048
:1014940083160313E8000030E900EC0A1430EA0074
:1014A4000030EB00831203179001910103134208EB
:1014B400031D5E2ACB0AC20183166C080319722D20
:1014C40083160430570783120317A90083160313E6
:1014D40058080318013E83120317AA001608AB002C
:1014E4001508AC008A1184238A1503171408B30065
:1014F4008A11DF208A1503171308B3008A11DF202D
:101504008A1503171A08B3008A11DF208A150317F6
:101514001908B3008A11DF208A1503171808B300CD
:101524008A11DF208A1503171708B3008A11DF20F8
:101534008A150C308316570783120317B3008316DA
:10154400031358080318013E83120317B4008A11C9
:1015540082208A150F3070050317B5008316031314
:101564006A08F000F00D7010F00D7010700883120E
:101574000317B5040C30831603135707831203179C
:10158400B3008316031358080318013E831203178C
:10159400B4008A11B1208A150D30831657078312BF
:1015A4000317B3008316031358080318013E83126C
:1015B4000317B4008A1182208A15C03070050317FE
:1015C400B50083160313680883120317B5040D309E
:1015D40083160313570783120317B30083160313E9
:1015E40058080318013E83120317B4008A11B1206E
:1015F4008A15003083166906031D022B1230680613
:10160400031D392B0E30570783120317A9008316C5
:10161400031358080318013E83120317AA00053068
:10162400AB00EE30AC008A1184238A151430831683
:10163400570783120317A9008316031358080318C6
:10164400013E83120317AA000230AB000430AC0041
:101654008A1184238A1505300317B3008A11DF2009
:101664008A1578300317B3008A11DF208A15831690
:10167400550883120317100783160313ED00831212
:10168400031711080318013E831603135607EE00CF
:101694006A08ED076B080318013EEE07831203176F
:1016A400120803195B2B8A119F278A158A11682750
:1016B4008A15BF300317A9001930AA008316031333
:1016C4006E0883120317AB00831603136D0883128D
:1016D4000317AC008A1184238A15C7300317A900A5
:1016E4001930AA00AB01AC018A1184238A15BD30DC
:1016F4000317A9001930AA0083160313550883128F
:101704000317AB0083160313560883120317AC00A8
:101714008A1183218A1516300317B3008A11D32046
:101724008A15700803179B001730B3008A11D32061
:101734008A1570080317AB00C730A9001930AA0036
:101744001B08AC008A1184238A1583166D08BD3EDC
:10175400E20019300318013E6E07E300103057070A
:1017640083120317A9008316031358080318013EB4
:1017740083120317AA00AB01AC018A1184238A15D2
:10178400013083166D05E100620883120317B3006C
:1017940083160313630883120317B400B5018A1177
:1017A400B1208A15C9300317A9001930AA00D13015
:1017B400AB001930AC00831603136108620783126F
:1017C4000317AD008316031363080318013E831245
:1017D4000317AE00AF018A1192238A1508308316CD
:1017E4000313620783120317A90083160313630804
:1017F4000318013E83120317AA008316031361081A
:1018040083120317A9070318AA0AAB010630AC0018
:101814008A1184238A150A308316620783120317F8
:10182400A9008316031363080318013E83120317E8
:10183400AA0083160313610883120317A907031868
:10184400AA0A1008831603136A07F3006B08031827
:10185400013E831203171107F4007408F000F1012C
:101864007008AB007308AC008A1184238A158316B0
:10187400570883120317A900831603135808831209
:101884000317AA001008831603136A0783120317A9
:10189400AB00831603136B080318013E831203176E
:1018A4001107AC000C30AB070318AC0A8316031302
:1018B400610883120317AB070318AC0A8A1183214A
:1018C4008A1516300317B3008A11D3208A157008BD
:1018D40003179B001730B3008A11D3208A157008B0
:1018E4000317AB0010308316031357078312031733
:1018F400A9008316031358080318013E8312031723
:10190400AA001B08AC008A1184238A150E308316A2
:101914006D0783120317A900831603136E080318B7
:10192400013E83120317AA008A11D0218A15831657
:101934006F080319392D1030E8000030E900EF0179
:101944008312031792010230B800831603136A0846
:10195400570783120317B900831603135808031893
:10196400013E6B0783120317BA008A112E208A15D1
:101974000E3083165307831203179C008316031338
:1019840054080318013E831203179D0083160313A2
:101994005508831203179C0783160313560803186C
:1019A400013E831203179D07831603136A088312EB
:1019B40003179C07831603136B080318013E831255
:1019C40003179D078A11BB278A15CB0ABE3003175C
:1019D4009C00831603136608831203179D00831665
:1019E40003136708831203179E0083160313640806
:1019F400831203179F0083160313650883120317CA
:101A0400A0000E3003136D020317A1000030031C65
:101A1400013E03136E020317A20083160313550835
:101A240083120317A102031CA2038316031356088F
:101A340083120317A202831603136A08831203177F
:101A4400A102031CA203831603136B08831203175A
:101A5400A2026430A3008A1173258A1570089000CD
:101A64007108910003136418382DCB01622A831284
:101A74004B080319722D03171008F0001108F10028
:101A8400F201F3011308F00714080318140FF10707
:101A940015080318150FF20716080318160FF30795
:101AA40070089300710894007208950073089600FA
:101AB400113083160313E8000030E9008312CB01D0
:101AC40003179201143083160313EA000030EB006D
:101AD400831203179001910101300313C200622A9B
:021AE4000800F8
:101AE6001F3083120317B3000130B4008A11C520DA
:101AF6008A151F300317B3000230B4008A11A320E1
:101B06008A15143003179C00831603135308831297
:101B160003179D008A1184278A158A1192278A1530
:101B260016309C00831603135508831203179D0075
:101B36008A1184278A158A1192278A1517309C00E4
:101B4600831603135408831203179D008A118427F2
:0A1B56008A158A1192278A150800EB
:101B60001F3083120317B3000130B4008A11C5205F
:101B70008A151F300317B3000230B4008A11A32066
:101B80008A15143003179C0083160313530883121D
:101B900003179D008A1184278A1512300317B3009A
:101BA0000130B4008A11A3208A158A1192278A1560
:101BB0001230B3000130B4008A11C5208A151630E6
:101BC0000317B3008A11D3208A15831655088400A1
:101BD00070088000173083120317B3008A11D320D6
:0E1BE0008A15831654088400700880000800DF
:101BEE00C43083120317B3001930B4008A11822057
:101BFE008A1570088316D300642ED530831203170E
:101C0E009C0019309D0069309E0004309F0000201A
:101C1E007008003A031D632EC430B3001930B400AF
:101C2E000230B5008A11B1208A158A119F278A15B4
:101C3E00CB300317A9001930AA00CF30AB001930F2
:101C4E00AC00D530AD001930AE00AF018A11922331
:101C5E008A15CB30A9001930AA006930AB000430C8
:101C6E00AC000030AD008A11AE218A15C5300317C5
:101C7E00A9001930AA00CB30AB001930AC00CF3020
:101C8E00AD001930AE00AF018A1192238A15C5300E
:101C9E00A9001930AA005E30AB000630AC0000304F
:101CAE00AD008A11AE218A153C300317A900003011
:101CBE00AA008A11D0218A156A2E8316031353089F
:081CCE00013A0319042E08007D
:101CD60083160313560883120317B30083160313E0
:101CE600570883120317B4008A1182208A157008D8
:101CF6008316E1008A1122238A1570088316E000F4
:101D06008A1122238A1570088316DF008A1122237E
:101D16008A1570088316DE0000305F06031D952EB7
:101D260000305E06031D982E592F8A1122238A152C
:101D360070088316E3008A1122238A157008831619
:101D4600E200BE30831203179C00C9309D00193093
:101D56009E0004309F000030A0008A113F258A159E
:101D660002300317B8000830831603135607831290
:101D76000317B9008316031357080318013E83128D
:101D86000317BA008A112E208A150E3083165307C0
:101D9600831203179C008316031354080318013E8D
:101DA600831203179D008316031355088312031726
:101DB6009C0703189D0A08309C0703189D0A8A1180
:101DC600BB278A15BE3003179C00831603136008D1
:101DD600831203179D0083160313610883120317EA
:101DE6009E00831603135E08831203179F00831653
:101DF60003135F0883120317A0000830831603132A
:101E0600620283120317A1000030031C013E8316F1
:101E16000313630283120317A2006430A3008A111E
:101E26006E258A1570088316E2007108E3007008B3
:101E360071040319592FD830831203179C00B5304B
:101E46009D0019309E0006309F000030A0008A11C8
:101E56003F258A15D83003179C00BE309D00831697
:101E660003135E08831203179E00831603135F088D
:101E7600831203179F008316031360088312031748
:101E8600A00083160313610883120317A1008316AB
:101E96000313620883120317A20083160313630851
:0E1EA60083120317A3008A113B248A1508003B
:101EB40083120313EF011F300317B3000130B40082
:101EC4008A11A3208A151F300317B3000230B4000F
:101ED4008A11C5208A1519300317B3008A11D3203B
:101EE4008A157008003C0318802F8A110A160020F6
:101EF4008A150A12831203137008EF001F300317A8
:101F0400B3000130B4008A11C5208A151F300317AD
:101F1400B3000230B4008A11C5208A156F08F0009E
:021F24000800B3
:101F26008A1194208A150A128000840AC20A0319AB
:0A1F3600C30AF003031D932F0800F7
:101F40008A110A1668278A150A128312031385015B
:101F5000FF308316850083128601FF3083168600CA
:101F600083128801831688018A11F2278A15283086
:101F70008316C4002430C5000130C6008A110A1639
:0C1F8000F6238A150A125A27C32FC52F1A
:1020000083160313D00183126414E4101F300317E6
:10201000B3000130B4000A12C5200A161F3003179E
:10202000B3000230B4000A12C5200A160317B80123
:10203000031343080317B900031344080317BA0036
:102040000A122E200A1687103A300317BB000A1214
:1020500003200A160317BB010A1203200A16700890
:10206000C3000317BB010A1203200A167008C4003C
:102070000317BB010A1203200A167008ED000317AC
:10208000BB010A1203200A167008EE000317BB01F9
:102090000A1203200A1670088316CE008312031753
:1020A000BB010A1203200A1670088316CF008312A0
:1020B00087140430ED02031CEE034408193C031D91
:1020C00063284308AD3C031C772843187728831600
:1020D000CF1B772883126E08053C031D71286D08FD
:1020E000EE3C031C77288316CE1F77287A28013010
:1020F000F000ED2A83120317B3010A12D3200A1647
:1021000070088316CC00013083120317B3000A1243
:10211000D3200A1670088316CD004C0883120317CB
:10212000A900831603134D0883120317AA00031393
:102130006D0883164C0783120317AB008316031335
:102140004D080318013E83126E070317AC00AF3031
:10215000AD001930AE000130AF000A1292230A160A
:10216000BB30B3001930B4000A1282200A1670087E
:102170008316CF000A1222230A1670088316CE0097
:102180004F08083A031DC62806304E06031DE128F5
:10219000BD30831203179C0019309D003A309E0019
:1021A00007309F008A150A1200208A110A1670084B
:1021B000003A031DE0288A150A12F7258A110A162B
:1021C000B42A831603134F08083A031DE928003088
:1021D0004E06031DB02ACD30831203179C00193020
:1021E0009D0045309E0004309F008A150A12002091
:1021F0008A110A167008031DFF280313E414CD305A
:1022000003179C0019309D0069309E0004309F0028
:102210008A150A1200208A110A1670080319172954
:102220000313E418172902308316D000AF2ABD30FB
:1022300083120317B3001930B4000A1282200A1661
:10224000F0307005F1007108403A03192B29033072
:102250008316D000AF2ABD3083120317B3001930A4
:10226000B4000A1282200A1670088316CA00CB0135
:102270000F30CA050030CB05CA0DCB0D4A10CA0D70
:10228000CB0D4A10C33083120317B3001930B400CA
:102290000A1282200A16BF307005F1007108003A58
:1022A000031DAF2AC4300317B3001930B4000A125B
:1022B00082200A167008003A031DAF2A83164A08C6
:1022C000BD3EC80019300318013E4B07C900C63097
:1022D00083120317B3001930B4000A1282200A16C1
:1022E00070088316C7007008013A031D5C2A48086D
:1022F00083120317B30083160313490883120317CD
:10230000B4000A1282200A167008083A031D5B2ADC
:1023100083164808013E83120317B30000300318E8
:10232000013E83160313490783120317B4000A12F0
:1023300082200A167008003A031D5B2A831648089B
:1023400083120317B300831603134908831203177C
:10235000B400B5010A12B1200A160A129F270A1604
:102360000A1268270A16C7300317A9001930AA00F5
:10237000AB01AC010A1284230A16BD300317A90071
:102380001930AA00831603134A0883120317AB00FF
:10239000831603134B0883120317AC000A12832120
:1023A0000A1616300317B3000A12D3200A16700853
:1023B0008316D100173083120317B3000A12D320FB
:1023C0000A1670080317AB00C730A9001930AA001D
:1023D00083160313510883120317AC000A128423D7
:1023E0000A1602308316480783120317A9008316C2
:1023F000031349080318013E83120317AA00AB0117
:10240000AC010A1284230A168316480883120317A4
:10241000A90083160313490883120317AA00831621
:1024200003134A0883126D020317AB0083160313CC
:102430004B08031C013E83126E020317AC000E30E2
:10244000AB02031CAC030A1283210A1616300317D1
:10245000B3000A12D3200A1670088316D100173071
:1024600083120317B3000A12D3200A167008031749
:10247000AB00023083160313480783120317A90029
:102480008316031349080318013E83120317AA0099
:1024900083160313510883120317AC000A12842316
:1024A0000A166D080317A90003136E080317AA0084
:1024B0000A12D0210A16AF2A83164708113A031DC3
:1024C000712A4C08D3004D08D4004A08D5004808AA
:1024D000D6004908D7008A150A126B268A110A16F7
:1024E000AF2A831603134708063A031DAF2A10309C
:1024F0004C0783120317B300831603134D08031808
:10250000013E83120317B4000A1282200A167008D3
:102510008316D200D1010A1222230A1670088316EC
:1025200051078312ED00831652080318013E8312EF
:10253000EE000E30ED070318EE0A83164C08D300A8
:102540004D08D4004A08D5004B08D6004808D700EB
:102550004908D8008A150A1242208A110A16B42A9C
:10256000043083160313D0001E3083120317B30008
:102570004030B4000A12A3200A1601304302F100D1
:102580000030031C013E4402F2007208193C031D96
:10259000CB2A7108AD3C0318D82A0C300317B800B9
:1025A000AD30B9001930BA000A122E200A16EA2AF4
:1025B0000C300317B8000130031343020317B900AE
:1025C0000030031C013E031344020317BA000A1231
:0C25D0002E200A1683165008F0000800A8
:1025DC00831203179C018316031347080319F92A66
:1025EC000D30F000FB2A0530F00070088312031741
:1025FC009D000A1284270A16023003179C008316CA
:10260C000313470803190D2B3130F0000F2B30301A
:10261C00F0007008831203179D000A1284270A1613
:10262C000A300317B800EE30B9000530BA000A12B0
:10263C002E200A16043003179C0083160313470838
:10264C0003192B2B1530F0002D2B1230F0007008D5
:10265C00831203179D000A1284270A1606300317EB
:10266C009C0012309D000A1284270A168316470814
:10267C00031D492B0730831203179C000C309D005F
:10268C000A1284270A1683164708031D562B093095
:10269C00831203179C003F309D000A1284270A16F0
:1026AC0083121F300317B3000130B4000A12A320A9
:1026BC000A161F300317B3000230B4000A12A3200D
:1026CC000A16043003179C0003135E0803179D00C1
:1026DC000A1284270A16053003179C0003135F089F
:1026EC0003179D000A1284270A16023003179C0058
:1026FC000313600803179D000A1284270A1603307F
:10270C0003179C000313610803179D000A1284270A
:10271C000A1603179C010313620803179D000A1283
:10272C0084270A16013003179C0003136308031750
:10273C009D000A1284270A16153003179C009D0170
:10274C000A1284270A1612300317B3000A12D32078
:10275C000A167008E8008316D301C830D400C930BB
:10276C00D5008A150A12B0258A110A16D301FE303B
:10277C004805D40047080319C62B0130F000C72BBD
:10278C00F0017008D4044908D5008A150A12732583
:10279C008A110A16103083160313D3000130D400AB
:1027AC00D5018A150A1273258A110A161F30B30037
:1027BC000430B4000A12A3200A160A1292270A1631
:1027CC001F30B3000130B4000A12C5200A161F30A6
:1027DC000317B3000230B4000A12C5200A16080011
:1027EC0083160313071083120714831687108312A2
:1027FC0087140A1292270A16031307140A12922737
:10280C000A16031307100A1292270A160313071449
:10281C000A1292270A1603138710FF300317BB0006
:10282C000A1203200A1687140A1292270A165E301F
:10283C0083160313C7004408C8000630C9000030D3
:10284C00CA000A12D2270A166930C7004508C80008
:10285C000430C9000030CA000A12D2270A161F30F1
:10286C0083120317B3000130B4000A12C5200A16F4
:10287C001F300317B3000230B4000A12C5200A1629
:10288C0008300317B800B901BA010A122E200A1633
:10289C000A300317B800AD30B9001930BA000A126B
:1028AC002E200A160C300317B800AD30B9001930C1
:1028BC00BA000A122E200A160317B801B901BA0180
:1028CC000A122E200A1604300317B800AE30B900D5
:1028DC001930BA000A122E200A161F300317B30043
:1028EC000130B4000A12C5200A161F300317B300BA
:1028FC000230B4000A12A3200A1683164608C70039
:04290C00EE220800AF
:102ED000203084002C3083120313F000C730831697
:102EE000C2000F30C3008A150A1293278A110A16EE
:022EF0000800D8
:041F8E00883414344B
:041F9200E7341934E3
:081F9600C034A8340034AA3461
:0C1F9E0000341434A534763419343F3478
:041FAA0000341834B3
:081FAE0000340034003400345B
:0C1FB60047344534543420342F340034B8
:101FC200003401340834003406340434003400345C
:021FD2000034D9
:041FD40000340034A1
:0C1FD800FF34FF34FF34FF34FF34FF34CB
:021FE4000034C7
:101FE60074346534783474342F3470346C3461341A
:0A1FF60069346E340A340A340034F2
:102910003C347434613462346C3465343E343C3459
:10292000743472343E343C34743464342034763439
:1029300061346C34693467346E343D3474346F34CC
:1029400070343E343C347434613462346C346534F5
:10295000203462346F3472346434653472343D34FC
:10296000313420347334743479346C3465343D3408
:10297000273466346F346E3474342D3473346934D0
:102980007A3465343A3432343034703478343B3409
:10299000203466346F346E3474342D3466346134CC
:1029A0006D3469346C3479343A3420347434653499
:1029B00072346D3469346E3461346C343B34273492
:1029C0003E343C34743472343E343C3474346834B1
:1029D000203463346F346C347334703461346E3447
:1029E0003D3432343E344134443443343C342F3467
:1029F000743468343E343C342F34743472343E348E
:102A00003C34743472343E343C34743464343E3474
:102A100041344E3432343C342F34743464343E34D4
:102A20003C34743464343E343C3473346334723430
:102A30006934703474343E3464346F3463347534C0
:102A40006D3465346E3474342E34773472346934B2
:102A500074346534283441344E34323429343B34B0
:102A60003C342F34733463347234693470347434C6
:102A70003E343C342F34743464343E343C342F348C
:102A8000743472343E343C34743472343E343C34E6
:102A9000743464343E3441344E3433343C342F3453
:102AA000743464343E343C34743464343E343C34E2
:102AB0007334633472346934703474343E3464343F
:102AC0006F34633475346D3465346E3474342E343D
:102AD00077347234693474346534283441344E3474
:102AE000333429343B343C342F34733463347234FC
:102AF0006934703474343E343C342F347434643468
:102B00003E343C342F34743472343E343C342F34ED
:102B10007434613462346C3465343E343C342F3464
:102B2000743464343E343C34743464343E343C3461
:102B30007434613462346C346534203462346F34FC
:102B400072346434653472343D3431342034733437
:102B5000743479346C3465343D34273466346F34DE
:102B60006E3474342D34733469347A3465343A34C1
:102B700032343034703478343B34203466346F343B
:102B80006E3474342D34663461346D3469346C348D
:102B900079343A3420347434653472346D346934A1
:102BA0006E3461346C343B3427343E343C347434FA
:102BB00072343E343C3474346834203463346F34BB
:102BC0006C347334703461346E343D3432343E349A
:102BD00050344F345234543442342034283449343D
:102BE0004E34293420343A3420343C347334633442
:102BF00072346934703474343E3464346F34633402
:102C000075346D3465346E3474342E3477347234E4
:102C1000693474346534283450344F345234543465
:102C2000423429343B343C342F34733463347234AB
:102C30006934703474343E343C342F347434683422
:102C40003E343C342F34743472343E343C34733468
:102C5000633472346934703474343E34763461349D
:102C6000723420347334743472342C3469343B3409
:102C70007334743472343D34273427343B3466342F
:102C80006F347234283469343D3430343B34693421
:102C90003C3438343B3469342B342B3429347B3482
:102CA0007334743472342B343D3427343C347434EC
:102CB00072343E343C3474346434203462346734C7
:102CC00063346F346C346F3472343D342334633482
:102CD000633463346334633463343E344234553490
:102CE000543454344F344E342034233427342B346A
:102CF00069342B3427343C342F34743464343E34F8
:102D000027343B3469346634283450344F345234D9
:102D1000543442342634283431343C343C3469341D
:102D2000293429347B347334743472342B343D3475
:102D300027343C347434643420346234673463346C
:102D40006F346C346F3472343D34673472346534AC
:102D500065346E343E344F344E3427343B347D3446
:102D600065346C34733465347B3473347434723446
:102D70002B343D3427343C3474346434203462348E
:102D8000673463346F346C346F3472343D3472346E
:102D9000653464343E344F344634463427343B344F
:102DA0007D347334743472342B343D3427343C34E2
:102DB0002F34743464343E343C342F3474347234DD
:102DC0003E3427343B347D3464346F34633475349B
:102DD0006D3465346E3474342E347734723469341F
:102DE00074346534283473347434723429343B3485
:102DF0003C342F3473346334723469347034743433
:042E00003E34003428
:102E040048345434543450342F3431342E3431341F
:102E1400203432343034303420344F344B340A3498
:102E240043346F346E34743465346E3474342D34F6
:0E2E340074347934703465343A342034003408
:102E420074346534783474342F34683474346D34A3
:082E52006C340A340A34003428
:102E5A00763461347234203450344F34523454341A
:062E6A0042343D34003447
:102E7000763461347234203450344F345234543404
:062E800044343D3400342F
:102E8600763461347234203441344E3433343D3434
:022E9600003406
:102E980076346134723420345234453451343D34FC
:022EA8000034F4
:102EAA00763461347234203441344E3432343D3411
:022EBA000034E2
:042EBC003B3400346F
:042EC0003B3400346B
:042EC4003B34003467
:042EC8003B34003463
:042ECC003B3400345F
:103000003C342F347434613462346C3465343E346F
:103010003C342F34743464343E343C34743464347B
:103020003E343C347434613462346C34653420345E
:1030300062346F3472346434653472343D34313404
:1030400020347334743479346C3465343D3427342B
:1030500066346F346E3474342D34733469347A3496
:1030600065343A3432343034703478343B3420347C
:1030700066346F346E3474342D34663461346D3498
:1030800069346C3479343A342034743465347234AD
:103090006D3469346E3461346C343B3427343E34DF
:1030A0003C34743472343E343C34743468342034E8
:1030B00063346F346C347334703461346E343D3443
:1030C00033343E3450344F34523454344434203446
:1030D00028344F3455345434293420343A3420348D
:1030E0003C347334633472346934703474343E3431
:1030F00064346F34633475346D3465346E347434D1
:103100002E3477347234693474346534283450344E
:103110004F3452345434443429343B343C342F3407
:103120007334633472346934703474343E343C34F0
:103130002F34743468343E343C342F347434723455
:103140003E343C34733463347234693470347434D0
:103150003E347634613472342034733474347234CF
:103160002C3469343B347334743472343D34273432
:1031700027343B3466346F347234283469343D3438
:1031800030343B3469343C3438343B3469342B3488
:103190002B3429347B347334743472342B343D34FF
:1031A00027343C34743472343E343C3474346434E4
:1031B00020346234673463346F346C346F34723467
:1031C0003D342334633463346334633463346334AD
:1031D0003E344C34453444342034233427342B34A7
:1031E00069342B3427343C342F34743464343E3403
:1031F00027343B3469346634283450344F345234E5
:10320000543444342634283431343C343C34693426
:10321000293429347B347334743472342B343D3480
:1032200027343C3474346434203462346734633477
:103230006F346C346F3472343D34793465346C34AB
:103240006C346F3477343E344F344E3427343B344F
:103250007D3465346C34733465347B347334743446
:1032600072342B343D3427343C3474346434203489
:103270006234673463346F346C346F3472343D3489
:1032800023343934393439343934393439343E34E7
:103290004F344634463427343B347D3473347434ED
:1032A00072342B343D3427343C342F34743464343A
:1032B0003E343C342F34743472343E3427343B343F
:1032C0007D3464346F34633475346D3465346E34F6
:1032D00074342E3477347234693474346534283459
:1032E00073347434723429343B343C342F347334A3
:1032F000633472346934703474343E343C342F3463
:103300007434613462346C3465343E343C342F346C
:10331000743464343E343C342F34743472343E3468
:103320003C342F347434613462346C3465343E344C
:103330003C3470343E34543468346934733420344B
:103340006934733420344834543454345034203481
:1033500072346534713475346534733474342034A4
:1033600023343C34733463347234693470347434C9
:103370003E3464346F34633475346D3465346E3484
:1033800074342E34773472346934743465342834A8
:1033900052344534513429343C342F34733463343B
:1033A00072346934703474343E343C3470343E3496
:1033B0003C342F3442344F34443459343E343C345A
:0E33C0002F34483454344D344C343E340034F1
:1033CE003C346D3465347434613420346834743470
:1033DE00743470342D346534713475346934763404
:1033EE003D34273472346534663472346534733444
:1033FE0068342734203463346F346E347434653457
:10340E006E3474343D342734313430343B347534B7
:10341E0072346C343D3468347434743470343A34E9
:10342E002F342F343134393432342E34313436345F
:10343E0038342E3430342E343134373430342F3453
:10344E0027343E343C34483454344D344C343E34BA
:10345E003C3448344534413444343E343C342F34C7
:10346E0048344534413444343E343C3442344F3491
:10347E00443459343E343C34683431343E34503460
:10348E0049344334203431343634463438343834C5
:10349E0037342034283438344D3448347A3429348F
:1034AE0020342B34203445344E34433432343834C3
:1034BE004A343634303420344D3469346E34693401
:1034CE0020345734653462342034533465347234C6
:1034DE007634653472342C343C3470343E3461347A
:1034EE0076346534633420344D3469346B3472343D
:1034FE006F3443342034503452344F3420347634C5
:10350E0035342E3436342E3431343C342F34683442
:10351E0031343E343C3470343E343C3461342034E7
:10352E0068347234653466343D342234683474340D
:10353E00743470343A342F342F346F346C3469341D
:10354E0076346934653472342E3466346F3475349F
:10355E0072346E34653474342E3466347234653499
:10356E0065342E34663472342F3465342E34683418
:10357E0074346D346C3422343E344E344F345434FF
:10358E004934433445343C342F3461343E343C3476
:10359E0070343E343C3470343E343C346134203428
:1035AE0068347234653466343D342F343E345234CC
:1035BE0065346C346F34613464343C342F3461348C
:1035CE003E343C3470343E343C34733463347234A1
:1035DE0069347034743420347334723463343D344B
:1035EE002F3473343E343C342F347334633472349A
:0A35FE006934703474343E34003434
:02400E004A2F37
:00000001FF
